:0300000002007289
:030003000200F9FF
:03000B000201E807
:03001300020104E3
:20001B000201D5476573636877696E6469676B656974736D65737365722056657273696F3A
:20003B006E20312E302020766F6D2030352E31302E32303031204B6C617573204C65696433
:20005B00696E67657220496E7465726E657420446F776E6C6F6164758170D2B1D2B4D2B0BE
:20007B00D2B7D2B57B017AF4782412027E8958885975500075511075520075530075541078
:20009B00755500755A007B007A00758922758C38858C8AC2B9C28CC2A9758D38858D8BC2F6
:2000BB00BBC28EC2ABD288D28AD2A8D2AAC289C28BD2AF9002DAE55093D2B5F590C2B01125
:2000DB00F4E55193D2B0F590C2B711F4E55293D2B7F590C2B511F401D17E2FDEFE22C2A888
:2000FB00C0E0E55AB40022210DC2AAC0E0E55AB400177B007A00D28CD2A9755A0175502E5B
:20011B0075512E75522ED0E032C28CC2A98B568A57A958A859C082C08351A4D083D082E875
:20013B00602BB4FF0221735109E5507046855150E5522410F551780AC082C08312027EAB70
:20015B0056AA5751A4D083D0828852218E755005755126755228217C75500F75510A75525D
:20017B0005755A00C2B17B277A00D28AD28ED2ABD0E032E554C394104009E551C394104020
:20019B002621A7E551C39410400221D3E550C3955340257012E551C39554401C7009E552CE
:2001BB00C3955540136011855053855154855255D2B0D2B7D2B5511F217CDA10DB0EC28E73
:2001DB00C2ABC289C28BD2A8D2AAD2B1320ABA001C0BBB001875500E75512A75522A755A13
:2001FB0000C28CC2A9C289C28BD2A8D2AA32C0F075F06484F550E5F075F00A84F55185F0A6
:20021B0052D0F022755B10755C80755D80755B10755C80755D80D55DFDB2B4D55CF5D55B9E
:20023B00EF22E820E703C22122F404F8D22122EB20E703C22222D222EAF42401FAEBF43497
:20025B0000FB222021042022052230220122E8F42401F8E9F43400F9EAF43400FAEBF43421
:20027B0000FB22C0F053D0E7513D514AE88AF0A4C0E0C0F0E88BF0A4D00028F9E435F0FA12
:20029B00D0007B00515ED0F0227F007E0075F010C3E833F8E933F9EE33FEEF33FFEEC39A7F
:2002BB00F582EF9BF583B35004AF83AE82EC33FCED33FDD5F0DAEDF9ECF8EFFBEEFA22812B
:2002DB00DD92D0CCE0A0D580C084A4A398A2A6015D12504C6020550040042423182226FFED
:0F02FB00BA8CACFFD9ABAEB886BE89B9FEFB7F1B
:00030A01F2
